:020000040800F2
:100000000080012039230008892300088923000883
:1000100089230008892300088923000800000000C4
:10002000000000000000000000000000892300081C
:10003000892300080000000089230008E31F00084E
:1000400089230008892300088923000889230008E0
:1000500089230008892300084D2000085320000848
:10006000592000085F200008652000088923000847
:1000700089230008892300088923000889230008B0
:100080008923000889230008892300080000000054
:100090000000000000000000000000006B200008CD
:1000A00009250008A924000819250008892300084B
:1000B000C9240008D9240008E9240008D52500082F
:1000C000E1250008ED250008F9250008892300082E
:1000D0008923000859270008712700080000000044
:1000E000812000082D23000889230008000000005B
:1000F000000000000000000000000000892300084C
:100100000000000089230008F92400088923000862
:1001100000000000000000000000000000000000DF
:1001200089230008892300088923000889230008FF
:10013000892300080000000000000000000000000B
:1001400000000000000000000000000089230008FB
:1001500089230008892300088923000889270008CB
:10016000052600081126000800000000000000001D
:10017000000000000000000000000000000000007F
:1001800000000000892300080000000000000000BB
:0401900089230008B7
:1001940010B5054C237833B9044B13B10448AFF3BD
:1001A40000800123237010BD2800002000000000FF
:1001B400182900080C4B43B10C480D4910B5AFF396
:1001C40000800C48036823B910BD0A48036833B99A
:1001D4007047094B002BF7D0BDE810401847064B79
:1001E400002BF5D0184700BF0000000018290008B4
:1001F4002C000020280000200000000053B94AB958
:10020400002908BF00281CBF4FF0FF314FF0FF301A
:1002140000F07AB9ADF1080C6DE904CE00F006F8EF
:10022400DDF804E0DDE9022304B070472DE9F0476E
:100234008C460D460446089E002B51D18A4217462F
:100244006DD9B2FA82FEBEF1000F0BD0CEF1200CB4
:1002540001FA0EF520FA0CFC02FA0EF74CEA050C32
:1002640000FA0EF44FEA174A250CBCFBFAF81FFA01
:1002740087F90AFB18CC45EA0C4508FB09F3AB42A5
:100284000AD9ED1908F1FF3280F02381AB4240F224
:100294002081A8F102083D44ED1AA4B2B5FBFAF09E
:1002A4000AFB105544EA054400FB09F9A14509D9A4
:1002B400E41900F1FF3380F00A81A14540F207817F
:1002C40002383C44A4EB090440EA08400021002E13
:1002D40061D024FA0EF4002334607360BDE8F08723
:1002E4008B4207D9002E54D0002186E8210008460D
:1002F400BDE8F087B3FA83F1002940F08E80AB4269
:1003040002D3824200F2FA80841A65EB03050120CD
:10031400AC46002E3FD086E81010BDE8F08712B935
:100324000127B7FBF2F7B7FA87FEBEF1000F34D10D
:10033400EB1B3A0C1FFA87FC0121B3FBF2F8250CE6
:1003440002FB183345EA03450CFB08F3AB4207D91B
:10035400ED1908F1FF3002D2AB4200F2D1808046A1
:10036400ED1AA3B2B5FBF2F002FB105543EA0544C3
:100374000CFB00FCA44507D9E41900F1FF3302D2B9
:10038400A44500F2B8801846A4EB0C0440EA0840E7
:100394009DE731463046BDE8F087CEF1200405FAEA
:1003A4000EF307FA0EF720FA04F83A0C25FA04F4CF
:1003B40048EA0308B4FBF2F14FEA184502FB114482
:1003C4001FFA87FC45EA044501FB0CF3AB4200FA33
:1003D4000EF409D9ED1901F1FF3080F08A80AB42A7
:1003E40040F2878002393D44EB1A1FFA88F5B3FBCB
:1003F400F2F002FB103345EA034500FB0CF3AB4279
:1004040007D9ED1900F1FF386FD2AB426DD902382C
:100414003D44EB1A40EA01418FE7C1F1200722FA7B
:1004240007F88B4005FA01F448EA030320FA07FEB3
:100434004FEA134CFD404EEA040EB5FBFCF94FEABB
:100444001E440CFB19551FFA83F844EA054509FBC1
:1004540008F4AC4202FA01F200FA01FA08D9ED18E4
:1004640009F1FF3043D2AC4241D9A9F102091D443C
:100474002D1B1FFA8EFEB5FBFCF00CFB10554EEA4B
:10048400054400FB08F8A04507D9E41800F1FF353E
:1004940029D2A04527D902381C4440EA0940A4EBDC
:1004A4000804A0FB02894C45C6464D4615D312D01C
:1004B40056B1BAEB0E0364EB050404FA07F7CB401C
:1004C4001F43CC40376074600021BDE8F0871846B4
:1004D400F8E69046E0E6C245EAD2B8EB020E69EBD4
:1004E40003050138E4E72846D7E7404691E781460B
:1004F400BEE7014678E702383C4445E7084608E78A
:10050400A8F102083D442BE7704700BF01210D20EC
:1005140002F044B908B501210D2002F093F94FF41B
:100524007A7002F0B1F90D20002102F08BF94FF43A
:100534007A70BDE8084002F0A7B9000030B595B064
:100544000022274B0192196C41F0805119641B6CF5
:10055400244903F080530193019B02920B6823F416
:10056400404343F400430B600B680F9203F4404391
:100574000293029B01230B9310230C9310934FF4CB
:10058400A873022411930425072308A808940E9441
:100594001295139300F0B8FF00B1FEE70F23039305
:1005A40005904FF480530790214603A804940693C2
:1005B40001F05AF9044600B1FEE701F0EFF94FF4F7
:1005C4007A73B0FBF3F000F0F3F9284600F016FA62
:1005D400224621464FF0FF3000F0A8F915B030BD97
:1005E4000038024000700040B0F86A30013303F074
:1005F4003F03A0F86A30B0F86A30B0F868009BB2E4
:1006040098424FF0FF3018BF00207047B0F8F43024
:10061400B0F8F600181A00F03F007047B0F8F43054
:10062400B0F8F6209BB293421ABFD0F8F030985C31
:100634004FF0FF307047B0F8F420B0F8F63092B2C3
:100644009A421FBFD0F8F020D25C013303F03F037D
:100654001ABFA0F8F63010464FF0FF307047000084
:1006640010B5B0F8FC4001230374E31803F03F0312
:10067400B0F8FE2092B29342FAD0D0F8F820115587
:1006840000F19404A0F8FC30204601F0C5FF18B92D
:100694000249204601F0D2FF012010BDED050008FB
:1006A400037C33B1B0F8FC20B0F8FE309BB29A4220
:1006B400FAD1704700F11103C0F8F03000F1510293
:1006C4000023A0F8F430A0F8F630C0F8F820A0F821
:1006D400FC30A0F8FE30704738B5002343604FF477
:1006E4007A7383600F4B03600F4B984204460D46A8
:1006F4000BD10E4B1A785B7880F8ED2080F8EC3043
:100704002046FFF7D7FF204638BD0949284601F0A7
:10071400E7FD084984F8ED00284601F0E1FD84F87E
:10072400EC00EDE76C2B000844000020282B0008A7
:10073400982A0008E02A000801490248FFF7CCBFC4
:1007440000440040440000202DE9F04106460D46D7
:1007540001EB02080C464445A4EB050707D03368B7
:1007640014F8011B1B68304698470028F3D138461B
:10077400BDE8F08110B5044602F084F8E060236817
:100784002046DB689847002808DA02F07BF8E36823
:10079400C01AA3689842F2D34FF0FF3010BD2DE980
:1007A400F04180460D468F180C46BC42A4EB05066A
:1007B40007D04046FFF7DEFF002802DB04F8010BF8
:1007C400F3E73046BDE8F0812DE9F84380468946D9
:1007D40016461C467BB1D7181546AF42A5EB060456
:1007E40009D04046FFF7C6FF002804DB484502D085
:1007F40005F8010BF1E72046BDE8F883836810B5DE
:10080400044613B1032201469847204610BD000058
:1008140008B5044B2BB10448FFF7F8FE08B1AFF359
:10082400008008BD000000004400002001F0DFBB90
:100834007047704708B5032000F066F8BDE808402B
:10084400FFF7F4BF08B5FFF7F4FFFFF75FFE044CB2
:10085400FFF760FE002CFBD0FFF7DAFFF8E700BFDC
:10086400150800087047000038B50E4A0E4B0546BF
:1008740018784FF47A73B3FBF0F31068B0FBF3F01D
:1008840000F096F8044658B90F2D09D802462946B7
:100894004FF0FF3000F04AF8044B20461D6038BD8D
:1008A400012038BD2400002004000020080000209E
:1008B40008B50B4B1A6842F400721A601A6842F4C5
:1008C40080621A601A6842F480721A60032000F091
:1008D4001BF80F20FFF7C8FFFFF7C4FF002008BD77
:1008E400003C0240034A044B11681B780B4413601C
:1008F400704700BF0C04002004000020014B18685E
:10090400704700BF0C040020074AD36823F4E06357
:100914001B041B0C43F0BF63000243F4003300F4D8
:10092400E0600343D360704700ED00E0174B30B53F
:10093400DC68C4F30224C4F10703251D042B28BF7B
:100944000423062D4FF0010505FA03F303F1FF33E9
:100954008CBF033C00241940A14005FA04F4013C77
:100964002240002842EA01024FEA0212ADBF00F120
:10097400604000F00F00064B00F56140B5BFD2B2F5
:10098400D2B21A5480F8002330BD00BF00ED00E05D
:1009940014ED00E0002808DB4209012300F01F00E9
:1009A40003FA00F0014B43F82200704700E100E035
:1009B4000138B0F1807F0AD2064B074A5860F02113
:1009C40082F823100020072298601A6070470120E3
:1009D400704700BF10E000E000ED00E0002809DBF4
:1009E4004309012200F01F0002FA00F06033024ABA
:1009F40042F82300704700BF00E100E0044B1A688E
:100A040004280CBF42F0040222F004021A6070476A
:100A140010E000E0704708B5FFF7FCFF08BD90F850
:100A24003530022B03D080234365012070470268D0
:100A3400052380F83530136823F001031360002088
:100A44007047000008B5044B5969014202D058614F
:100A540001F0E4FA08BD00BF003C014037B590F84E
:100A64003D40282C34D1002930D0002A2ED090F8D3
:100A74003C40012C2CD00568012480F83C402C68B3
:100A8400E4075EBF2C6844F001042C602C6824F455
:100A940000642C60292480F83D40202480F83E40E6
:100AA400002404644285C362438D019403856B6909
:100AB4000193AB690193019B6B68416243F4E0636A
:100AC40080F83C406B60204603B030BD0120FBE75A
:100AD4000220F9E737B590F83D40282C34D100299D
:100AE40030D0002A2ED090F83C40012C2CD0056840
:100AF400012480F83C402C68E4075EBF2C6844F075
:100B040001042C602C6824F400642C602A2480F8EE
:100B14003D40202480F83E40002404644285C362A2
:100B2400438D019403856B690193AB690193019B28
:100B34006B68416243F4E06380F83C406B6020469C
:100B440003B030BD0120FBE70220F9E790F83D3007
:100B5400202B14D1282380F83D3003681A68D2076B
:100B64005EBF1A6842F001021A601A6842F4806299
:100B74001A605A6842F440725A600020704702209A
:100B840070477047704770477047704790F83D3022
:100B9400293B012B10B50368044639D800220263AF
:100BA400282280F83D201A6822F400621A605A68EC
:100BB40012F4006254D05A68606B22F400625A60E6
:100BC40090F83530012B394B31D00365FFF727FFFF
:100BD40050B12268606B136823F001031360202373
:100BE40084F83D30036D984794F83D30282B0ED19E
:100BF400236C5B070BD52E4BE36220220023236377
:100C0400204684F83D2084F83E3001F0AEFC10BD4F
:100C140090F83D20602A05D05A6812055CBF202256
:100C240080F83D200022226384F83E20BBE7A06BBD
:100C34000365FFF7F4FE0028D6D0226853695806EE
:100C440004D5636A1269591C61621A702268A06B28
:100C5400136823F001031360202384F83D30C1E7B7
:100C640094F83D10602914D1202184F83D102264A9
:100C74005A69510604D5626A1B69511C616213707A
:100C84002268136823F0010313602046FFF77DFFF9
:100C9400AAE75A69520604D5626A1B69511C61624B
:100CA4001370204601F08EFC9EE700BFC1140008BB
:100CB4000000FFFF0368F0B59D6959695A6890F810
:100CC4003E40E4B2102C8DB002D0402C40F055824E
:100CD40011F0011F66D0970564D590F83E40402C72
:100CE40043D1046D002C3BD1446C04F0FE041C6120
:100CF400984E994C2E400C40002E00F09F81974D49
:100D04000D40002D00F06681550540F16381002CF3
:100D140040F0608190F83D20058D90F83E10C46A43
:100D2400D2B2C9B2002D40F00581212A40F00481DD
:100D3400042C00F06C81082C00F0698114F5803FCC
:100D440000F065815A6822F4E0625A60112303635B
:100D540080F83E50202380F83D30FFF712FFF6E084
:100D6400446C44F00104E4B2C1E70469B4F5804F73
:100D740005D190F83D40212C446CF2D1B5E7046DC7
:100D840034B9446CE41104F0060444F0F004AEE712
:100D9400046D012CACD1446CE41104F0060444F05D
:100DA400F104A4E76E4C0C401CB1960501D5446CCB
:100DB400D9E76C4C0C40002C9AD0940598D590F847
:100DC4003E40C66AD0F830E090F83D70222FE4B27D
:100DD40040F0A880076D47B9402C06D101975C69A3
:100DE40001949C690194019C82E7046D8CB90769A4
:100DF400B7F5404F0DD102945C6902949C6902944A
:100E0400029C1C6844F480741C60046D0134046505
:100E14006EE7448DA4B254B903945C6903949C694D
:100E24000394039C1C6844F400741C6019E0448D12
:100E3400A4B2012C42D116F5803F1BD11C6824F4C6
:100E440080641C605C6814F400640CD01C6824F496
:100E540080641C60002404945C6904949C69049478
:100E6400049C0024D3E705945C6905949C6905946B
:100E7400059CD7E7042E15D0082E13D0BEF1120F0F
:100E840010D0C46A022C1C6814BF24F4806444F497
:100E940080641C60002406945C6906949C69069432
:100EA400069CDEE71C6824F480641C60002407941C
:100EB4005C6907949C690794079CB3E7448DA4B2CA
:100EC400022C1CD1C46A022C1C681DBF24F480644B
:100ED4001C601C6844F4806418BF44F400641C6003
:100EE4005C68270542BF5C6844F480545C6000245D
:100EF40008945C6908949C690894089CB1E71C6890
:100F040044F480641C605C68260542BF5C6844F459
:100F140080545C60002409945C6909949C69099478
:100F2400099C9EE700240A945C690A949C690A94CB
:100F34000A9CDDE6212A03D0402908D1222A06D1C1
:100F4400428D92B282B95A6822F480625A600DB01E
:100F5400F0BD00BF04001000040001008000010087
:100F6400080001000200010090F83E20402A27D129
:100F7400026D7AB9C26C012A826C05D1D2B21A61AF
:100F8400036D02330365E2E7C2F307221A61036DBE
:100F94000133F7E7026D012A02D1826CD2B2F5E780
:100FA400026D022AD3D190F83D20222A04D11A6876
:100FB40042F480721A60CAE790F83D20212AC6D113
:100FC400426A511C416212781A61438D013B9BB203
:100FD4004385BCE7002CBAD09405B8D5C16A90F813
:100FE4003D20212AB3D1428D92B2002AE8D10429AE
:100FF4000DD008290BD011F5803F08D0596821F491
:10100400E06159601123036380F83E20A2E65A6828
:1010140022F4E0625A601A6842F400721A600023F3
:101024002022036380F83D2090F83E2080F83E3073
:10103400402A7FF492AEFFF7A6FD88E7904D0D405D
:10104400002D41D051053FD5002C3DD190F83D20D5
:10105400222A7FF47CAF428D92B2032A13D9426ACA
:101064001B69511C41621370438D013B9BB2438544
:10107400438D9BB2032B7FF46AAF0268536823F459
:101084008063536063E7012A3FF661AF1A6822F474
:1010940080621A605A6822F4E0625A60426A1B69EC
:1010A400511C41621370438D013B9BB24385202345
:1010B40080F83D30046390F83E3080F83E40402B89
:1010C40058D1FFF761FD42E7002C3FF440AF97058C
:1010D4007FF53DAFC16A428D92B2042A426A08D1BB
:1010E400596821F480615960511C1B694162137075
:1010F4006BE7448DA4B2032C08D1596821F48061B4
:101104005960196821F480611960EDE7448DA4B237
:10111400022CE9D10139012919689DBF21F48061AC
:101124001960196841F4007198BF41F48071196025
:101134001B69511C41621370438D013B9BB2438573
:10114400436A5A1C4262026812691A70438D02682B
:10115400013B9BB24385536823F4407353602023BF
:1011640080F83D300023036390F83E2080F83E3041
:10117400402AA5E7FFF706FDE9E6424C0C4074B1AE
:1011840096050CD599699B6981F004011D06C1F38C
:10119400800154BF8289028B01F0C4F9D7E63A4C2E
:1011A4000C40002C74D0940572D590F83D205968F9
:1011B40021F4E061596000210B9159690B91196880
:1011C40041F0010119600B99196821F480611960DB
:1011D40059680905D2B20CD590F83D10222903D0E4
:1011E40090F83D102A2929D1816B0968496889B290
:1011F4004185418D89B2E1B159694F0708D5416AEA
:101204001B694C1C44620B70438D013B9BB24385AC
:1012140001684B695E0608D5436A09695C1C44622F
:101224001970438D013B9BB24385036C43F0040367
:101234000364036C23B1FFF7A9FC88E6416BD4E790
:10124400A2F1280102290AD8104AC26220220363AB
:1012540080F83D2080F83E3001F087F977E6036B93
:10126400222B02D0222A7FF472AE002320220363B1
:1012740080F83D2080F83E3001F08EF967E600BF2B
:101284004000010002000100100001000000FFFF07
:10129400394E3A4C2E400C40002E36D0384D0D407D
:1012A4003DB3550525D524BB90F83D10428D92B22F
:1012B400C9B2002A3FF44BAE426A541C446212780D
:1012C4001A61428D013A92B24285428D92B2002A4D
:1012D4007FF43DAE29297FF43AAE5A6822F4806245
:1012E4005A6021230363282380F83D3001F066F916
:1012F4002DE6002C3FF42BAE94057FF528AE428DED
:1013040092B2002A7FF45CAE21E61E4D0D4035B347
:10131400510524D51CBB90F83D20418D89B2D2B231
:1013240000293FF414AE416A1B694C1C44620B70E3
:10133400438D013B9BB24385438D9BB2002B7FF4CD
:1013440006AE2A2A7FF403AE0268536823F480634E
:10135400536022230363282380F83D308CE7002C5C
:101364003FF4F5AD92057FF5F2AD428D92B2002ABD
:101374003FF4EDAD426AB7E604001000040001003A
:101384008000010040000100F8B50368494A5E6925
:101394005D681642044608D0E80506D5226C42F082
:1013A400010222646FF480725A6116F4813F08D0FE
:1013B400E90506D5226C42F0020222646FF4007241
:1013C4005A6116F4823F36D0EA0534D594F83E705B
:1013D400618D94F83D20206B202F89B2D2B258D170
:1013E400002956D102F0F701212903D0282A50D12F
:1013F40021284ED194F83D20E16A0429D2B201D0CB
:1014040008292CD1282A2AD12B4AE2625A6822F4CC
:10141400E0625A606FF480625A611A6822F4806252
:101424001A60002320222363204684F83D2084F898
:101434003E3001F09AF816F4843F09D0EB0507D545
:10144400236C43F00803236423686FF400625A6139
:10145400236C73B32046BDE8F840FFF797BB212AFD
:1014640023D11549E1622263202284F83D20002221
:1014740084F83E205A6822F4E0625A606FF4806275
:101484005A611A6822F480621A60204601F096F8C4
:10149400D1E7226C42F00402226494F83E20102A20
:1014A40002BF1A6842F400721A606FF480625A61D3
:1014B400C1E7F8BD000101000000FFFF806B08B523
:1014C4000368416B1A6822F480621A600022428524
:1014D4000A65816B0A6590F83D1060294FF0200180
:1014E40080F83D1080F83E2007D102641A6822F08B
:1014F40001021A60FFF749FB08BD1A6822F00102D5
:101504001A6001F05FF808BD2DE9F341044618B9EB
:10151400012002B0BDE8F0810368DD0710D4236820
:10152400980758D423681A0700F19A8023685B0748
:1015340000F1B880A269002A40F019810020E8E790
:10154400A64B9A6802F00C02042A07D09A6802F0AB
:101554000C02082A0AD15B68590207D59F4B1B6805
:101564009A03DCD56368002BD9D1D1E763689B4D1E
:10157400B3F5803F11D12B6843F480332B60FFF720
:10158400BDF9964D06462B689B03C8D4FFF7B6F900
:10159400801B6428F7D90320BBE7B3F5A02F04D13F
:1015A4002B6843F480232B60E5E72A6822F4803219
:1015B4002A602A6822F480222A60002BDFD1FFF7F8
:1015C4009DF906462B689F03A9D5FFF797F9801B61
:1015D4006428F7D9DFE7814B9A6812F00C0F07D023
:1015E4009A6802F00C02082A11D15B685E020ED4DC
:1015F4007A4B1A68950702D5E268012A88D11A68DD
:10160400216922F0F80242EAC1021A608AE7E2681C
:10161400734BB2B101221A60FFF770F96F4D0646A1
:101624002B68980707D52B68226923F0F80343EA4F
:10163400C2032B6076E7FFF761F9801B0228EFD91C
:10164400A9E71A60FFF75AF9644D06462B68990713
:101654007FF568AFFFF752F9801B0228F6D99AE7A5
:101664006269604B7AB101221A60FFF747F95B4D5A
:1016740006466B6F9F073FF559AFFFF73FF9801B95
:101684000228F6D987E71A60FFF738F9534D064662
:101694006B6F98077FF54AAFFFF730F9801B02287C
:1016A400F6D978E74D4B1A6C12F0805228D101928A
:1016B4001A6C42F080521A641B6C03F0805301933D
:1016C400019B0126484D2B68D9051BD5A368434DC2
:1016D400012B27D12B6F43F001032B67FFF70EF982
:1016E4003E4D074641F288382B6F9B0739D5002EB3
:1016F4003FF420AF394A136C23F08053136419E785
:101704000026DFE72B6843F480732B60FFF7F6F8BD
:1017140007462B68DA05D9D4FFF7F0F8C01B022876
:10172400F7D938E7052B04D12B6F43F004032B675B
:10173400D0E72A6F22F001022A672A6F22F00402FE
:101744002A67002BCAD1FFF7D9F841F28838074637
:101754002B6F9807CBD5FFF7D1F8C01B4045F7D9BD
:1017640019E7FFF7CBF8C01B4045BDD913E71B4D64
:10177400AB6803F00C03082B3FF4CAAE1B4E0023E6
:10178400022A336034D1FFF7B9F807462B68990170
:101794001ED4226AE3691343626A43EA8213E26A4B
:1017A40043EA0263A26A0D4C5208013A43EA024337
:1017B4006B6001233360FFF7A1F8054623689A01A3
:1017C4003FF5BCAEFFF79AF8401B0228F6D9E2E6D3
:1017D400FFF794F8C01B0228D8D9DCE60038024091
:1017E40000004742800E47420070004060004742BC
:1017F400FFF784F804462B689B017FF59FAEFFF743
:101804007DF8001B0228F6D9C5E600BF134908B5C8
:101814008B6803F00C03042B03D0082B03D010486F
:1018240008BD104808BD4A684B68496813F4800332
:1018340014BF0C480A48C1F3881118BF002302F0F2
:101844003F02A1FB0001FEF7D9FC044B5B68C3F324
:10185400014301335B00B0FBF3F008BD00380240E4
:101864000024F40000127A002DE9F0410D460446EC
:1018740010B90120BDE8F081444B1A6802F00F0250
:101884008A4228D321688F072DD4C80740D43F4B00
:101894001A6802F00F02954266D3226851076CD48D
:1018A400130707D53A4A2169936823F4604343EA4E
:1018B400C1039360FFF7AAFF354B364A9B68C3F315
:1018C4000313D35CD840344B18600F20FEF7CCFFD1
:1018D4000020BDE8F081CAB21A701B6803F00F0340
:1018E4009942C6D1CEE72A4B11F0040F1EBF9A6865
:1018F40042F4E0529A600E0742BF9A6842F4604292
:101904009A609A68A06822F0F00202439A60BCE7E9
:1019140062681F4B012A1DD11B6813F4003FA8D035
:101924001B4EB36823F003031343B360FEF7E6FFD3
:1019340041F288380746B368626803F00C03B3EBDE
:10194400820FA4D0FEF7DAFFC01B4045F3D9032071
:10195400BDE8F081911E01291B6802D813F0007FB5
:10196400DDE713F0020FDAE7EAB21A701B6803F03E
:101974000F039D427FF47DAF8FE70549E0688B68D4
:1019840023F4E05303438B608AE700BF003C02402A
:1019940000380240282C000824000020014B18685D
:1019A400704700BF240000200368DA68D20510B530
:1019B40004460AD59B68D90407D500F0A9FC22681F
:1019C400D368DBB263F4C073D3602368DA6892052A
:1019D4000BD59B689B0408D5204600F00FF82268BD
:1019E400D368DBB263F42073D360034B4FF400324B
:1019F4005A610123637710BD003C01407047022304
:101A040010B580F839300368196A41F21112114295
:101A1400044608D1196A40F24442114202BF1A68CE
:101A240022F001021A60204600F0AAFA002084F88D
:101A3400390084F8380010BD704770477047036858
:101A44001A69910710B504460ED5DA6892070BD5CA
:101A54006FF002021A619B6901229B07027677D01C
:101A6400FFF7EAFF0023237623681A69500710D58D
:101A7400DA6851070DD56FF004021A619B690222DE
:101A840013F4407F2276204668D0FFF7D5FF002369
:101A9400237623681A6912070FD5DA6810070CD564
:101AA4006FF008021A61DB69042299072276204646
:101AB4005AD0FFF7C1FF0023237623681A69D206A0
:101AC40010D5DA68D0060DD56FF010021A61DB6903
:101AD400082213F4407F227620464BD0FFF7ACFF58
:101AE4000023237623681A69D10708D5DA68D20758
:101AF40005D56FF001021A61204600F0CCFC236882
:101B04001A69100608D5DA68110605D56FF0800247
:101B14001A61204600F0A4F823681A69520608D511
:101B2400DA68500605D56FF040021A612046FFF7C7
:101B340085FF23681A69910622D5DA6892061FD5B3
:101B44006FF0200220461A61BDE8104000F087B80B
:101B540000F098FC2046FFF770FF83E700F092FC4A
:101B64002046FFF76AFF92E700F08CFC2046FFF75F
:101B740064FFA0E700F086FC2046FFF75EFFAFE7B6
:101B840010BD036A10B501248C4023EA04030362E8
:101B9400036A8A401A43026210BD000010B504466D
:101BA40000220068FFF7EDFF2368124A93420DD12B
:101BB400196A41F21112114208D1196A40F24442E1
:101BC400114202BF5A6C22F400425A64196A41F26B
:101BD4001112114208D1196A40F24442114202BF63
:101BE4001A6822F001021A60012384F839300020B7
:101BF40010BD00BF00000140036A10B504248C40EE
:101C040023EA04030362036A8A401A43026210BD92
:101C140010B5044600220068FFF7EEFF2368196A36
:101C240041F21112114208D1196A40F244421142A0
:101C340002BF5A6C22F400425A64196A41F211122A
:101C4400114208D1196A40F24442114202BF1A6893
:101C540022F001021A60002010BDFFF7D9BF7047BF
:101C640070470368DA6822F49072DA605A6922F0E5
:101C740001025A61202380F83A30704790F83930D5
:101C8400202B18D1A9B1A2B190F83830012B12D071
:101C9400C2840162828400230168C363212280F824
:101CA4003920CA6880F8383042F08002CA60184689
:101CB4007047012070470220704790F83A30222B79
:101CC40010B532D1836801690268B3F5805F836A15
:101CD4001FD15268C9B9C2F3080223F8022B8362E8
:101CE400C48D013CA4B2C4856CB90368DA6822F4DB
:101CF4009072DA605A6922F001025A61202380F856
:101D04003A3000F0D9FC002010BDD2B223F8012BE8
:101D1400E5E721B9591C526881621A70E0E75268FC
:101D2400591C816202F07F02F7E7022010BD000017
:101D340003681A68D96870B5160704465D6907D147
:101D440096065AD58D0658D5BDE87040FFF7B5BF45
:101D540015F0010502D111F4907F4ED0D30705D5BB
:101D6400CE0542BFE36B43F00103E363500704D5A0
:101D74001DB1E36B43F00203E363930704D51DB184
:101D8400E36B43F00403E363160704D51DB1E36B6F
:101D940043F00803E363E36B002B66D0950604D598
:101DA400880602D52046FFF788FF23685D69E26B49
:101DB4001107204602D415F040051AD0FFF751FF51
:101DC40023685A69520610D55A69606B22F04002A2
:101DD4005A6150B1254B0365FEF721FE002844D01B
:101DE400606BBDE87040036D1847204600F09EFC10
:101DF40070BD00F09BFCE56370BD160627D50D068B
:101E040025D594F83920212A2FD1A268B2F5805F14
:101E1400226A17D11188C1F308015960216979B97F
:101E240002322262E28C013A92B2E284EAB9DA68BE
:101E340022F08002DA60DA6842F04002DA6070BDB3
:101E44000132EEE7511C216212785A60EAE750062B
:101E54000BD54A0609D5DA6822F04002DA6020235D
:101E640084F83930204600F03BFC70BD751E000834
:101E740008B5806B0023C385C38400F057FC08BDFC
:101E840090F8392090F83A001043704786B0002348
:101E9400052853D8DFE800F003111E2B38450093C2
:101EA400274B28481A6B42F001021A631B6B03F09C
:101EB40001030093009B06B070470193204B224816
:101EC4001A6B42F002021A631B6B03F002030193C4
:101ED400019BF0E702931A4B1C481A6B42F0040270
:101EE4001A631B6B03F004030293029BE3E703935F
:101EF400134B17481A6B42F008021A631B6B03F06A
:101F040008030393039BD6E704930D4B11481A6B04
:101F140042F010021A631B6B03F010030493049B3A
:101F2400C9E70593064B0C481A6B42F080021A630A
:101F34001B6B03F080030593059BBCE70020BAE705
:101F44000038024000000240000402400008024041
:101F5400000C024000100240001C024008B5064973
:101F640000F0D0F9C0F3C430023802289ABF034B02
:101F7400185C002008BD00BF302900088C2B000825
:101F840000F028BA30B5124991B0054600F096F930
:101F94000190B8B12846FFF7E1FF1828044611D88C
:101FA4000C4BC340DB070DD50949284600F0AAF9BC
:101FB40010F4801F214601A806D0FFF74EFE01A8A9
:101FC400FFF71DFD11B030BDFFF7E8FDF7E700BFD7
:101FD4003029000811110001FEF790BC704708B5C4
:101FE400FEF780FCFEF717FDFFF7F8FF08BD08B504
:101FF400FEF75EFCBDE80840FEF7A0BA064838B517
:10200400A0F5A074A0F114051038FEF7F7FBA54263
:102014002846F7D138BD00BF8802002000230128DC
:1020240003F1010202D040081346F8E71421DBB2A1
:102034004B43044A181D1044816811B11A441369B2
:1020440018477047480100200120FEF7FBBC02201E
:10205400FEF7F8BC0420FEF7F5BC0820FEF7F2BC3E
:102064001020FEF7EFBC38B505242025A8B2FEF7F2
:10207400E9FC013C4FEA4505F8D138BD38B50624E2
:102084004FF48065A8B2FEF7DDFC013C4FEA45053C
:10209400F8D138BD224B234906221A7007221A753B
:1020A400082283F82820092283F83C200A2283F896
:1020B40050201722002083F8642083F8782083F8C6
:1020C4008C2083F8A02083F8B420282283F8C82029
:1020D40083F8DC2083F8F02083F8042183F81821A6
:1020E40083F82C21D860186258639864D8651867FF
:1020F400C3F88400C3F89800C3F8AC00C3F8C00068
:10210400C3F8D400C3F8E800C3F8FC00C3F8100116
:10211400C3F82401C3F83801034A00F0C3BB00BF6D
:1021240048010020012000080000002030B5C368E9
:1021340091FAA1F4B4FA84F491FAA1F10325B1FA65
:1021440081F1640005FA04F4490023EA040302FA65
:1021540001F11943C16030BD431C04D00C3111F9A5
:102164000C3C5A1C01D100207047984201F10C012B
:10217400F5D10120704700002DE9F041474B00F0F4
:102184000F08C0F3031401300E4601F0070753F89B
:10219400285003D14321424800F0F5F82046FFF7C8
:1021A40075FE0446826895FAA5F3B3FA83F395FAAB
:1021B400A5F103205B00B1FA81F100FA03F322EAEE
:1021C40003034A0000FA02F21343A360874236D89D
:1021D400DFE807F01D1D021DB8F1070FC6F3062046
:1021E40017D9626A2B0A93FAA3F1B1FA81F193FA2F
:1021F400A3F34FF00F0EB3FA83F389000EFA01F143
:102204009B0022EA010200FA03F3134363623B4694
:102214001AE0226A95FAA5F3B3FA83F395FAA5F1C5
:102224004FF00F0EB1FA81F19B000EFA03F389000F
:1022340022EA030200FA01F313432362E7E76A2167
:10224400174800F0A0F80023226895FAA5F0B0FA28
:1022540080F095FAA5F14FF0030EB1FA81F1400038
:102264000EFA00F0490022EA00028B40013F1343BA
:10227400012F236005D8636832074CBF2B43AB435F
:102284006360C6F30112012A02D0022A18BF002299
:1022940029462046BDE8F041FFF748BFE82B000877
:1022A4008F2B000891F900305A1C01D1002070478F
:1022B400834201D1486870470C31F3E7431C01D0D5
:1022C400FFF7F0BF002070474B6813B94FF0FF30A1
:1022D4007047834202D191F9000070470C31F3E753
:1022E40008B1FFF7F1BF4FF0FF30704791F90030AC
:1022F4005A1C01D118467047834201D1886870473F
:102304000C31F3E7431C01D0FFF7F0BF7047000026
:10231400034B1B6813B1034A10681847704700BF8A
:1023240088020020AC0200200148FFF73DBB00BF3B
:102334008C020020DFF834D0002103E00C4B5B5802
:10234400435004310B480C4B42189A42F6D30B4AC3
:1023540002E0002342F8043B094B9A42F9D300F00F
:1023640013F800F0B3FAFEF76DFA7047008001200D
:10237400B02C0008000000202800002028000020C5
:1023840010040020FEE7FEE70F49D1F8883043F43B
:102394007003C1F888300D4B1A68002042F0010226
:1023A4001A6098601A6822F0847222F480321A60EB
:1023B400074A5A601A6822F480221A60D8604FF0E3
:1023C40000638B60704700BF00ED00E000380240FE
:1023D400103000240368234A93420ED122494A6CE8
:1023E40022F001024A64214A934217D102F578424D
:1023F400536C23F4803353647047B3F1804F05D199
:1024040019490A6C22F001020A64ECE7184A934263
:102414000DD115490A6C22F002020A64154A93424E
:102424000DD102F57442536C23F40033E3E7124AEE
:1024340093420DD10C490A6C22F004020A640F4A3B
:102444009342D9D102F57042536C23F48023D2E72E
:102454000B4A9342C7D102F50B32136C23F00803E5
:1024640013647047000001400038024000400140FE
:1024740000040040004401400008004000480140BE
:10248400000C0040436C2BB1027E012A02D10021D2
:10249400043818477047034604381B6C03B11847C7
:1024A4007047000010B5064C206808B1FFF7C7FA62
:1024B400606A18B1BDE81040FFF7C1BA10BD00BF93
:1024C400B0020020024B586808B1FFF7B8BA704751
:1024D400B0020020024B986808B1FFF7B0BA704709
:1024E400B0020020024BD86808B1FFF7A8BA7047C1
:1024F400B0020020024B186908B1FFF7A0BA704778
:10250400B0020020024B186A08B1FFF798BA70476E
:10251400B0020020024B986A08B1FFF790BA7047E6
:10252400B0020020C3689A4210B504461CD171B9A8
:10253400436E80F8581003B1984794F8882004F14A
:10254400680120460823BDE81040FEF787BA00233F
:102554000122C36580F85820C16D0144022368310B
:10256400BDE81040FEF7B6BA10BD036E10B50446C0
:1025740043B190F85820012A04D1C26D12B1C16D43
:1025840068309847022384F858300023E3652046D6
:10259400BDE81040FEF7DABAC36D1F2BDEBFC36D72
:1025A4000133C36590F85820D2B2012A05D1C16D18
:1025B400014402236831FEF78DBA7047002380F886
:1025C4008830704790F859300BB9FEF7BFBA70479E
:1025D400014B1868FEF76EBB08030020014B186816
:1025E400FEF7D2BE08030020014B5868FEF762BB19
:1025F40008030020014B5868FEF7C6BE08030020FC
:10260400014B9868FEF756BB08030020014B9868FD
:10261400FEF7BABE0803002008B5074B90F8442023
:1026240053F82200FFF72CFC00F02100A0F1210355
:102634005842584108BD00BFB403002010B50446F9
:1026440000B390F84430104A42F823100F4A002196
:1026540042F82300022290F95A00FEF767F994F930
:102664005A00FEF797F9636EB4F86A1094F84400C0
:1026740013FA81F1064B012253F82000BDE8104003
:10268400FFF7FCBA10BD00BF640300208C030020D8
:10269400B403002010B548B10649002351F8234083
:1026A400A042DAB203D001330A2BF7D10A22104632
:1026B40010BD00BFB403002010B5FFF7EBFF0928DD
:1026C40008D8054B054A53F8203052F82000BDE8DD
:1026D4001040184710BD00BF140300203C03002025
:1026E40010B5FFF7D7FF092818D80D4B53F8204031
:1026F4000C4B53F820302046984701300ED0636EBF
:10270400B4F86A1094F8440013FA81F1064B0122DC
:1027140053F82000BDE81040FFF7B0BA10BD00BF69
:102724008C03002064030020B403002003681A68AB
:10273400D20782B002D55B68019308E01A6890075B
:10274400F9D41A685107F6D41A681207F3D4019B16
:1027540002B0704708B52520FEF740F9024B18680F
:10276400BDE80840FFF7E4BAB403002008B526200A
:10277400FEF734F9024B5868BDE80840FFF7D8BAB1
:10278400B403002008B54720FEF728F9024B586926
:10279400BDE80840FFF7CCBAB40300203A282DE97D
:1027A400F041884633D8224B1C56621C2FD0C4F308
:1027B4000315204E56F8253004F00F07FB40DB07C5
:1027C40010D51D492046FFF7C7FC10B12046FFF77E
:1027D400D9FB012303FA07F256F8253023EA020352
:1027E40046F82530B8F1050F1DD8DFE808F00318C6
:1027F4001214161A00212046FFF7BEFC0F490123CC
:1028040003FA07F251F82530134341F82530BDE8A7
:10281400F0811021EFE72021EDE70321EBE701210F
:10282400E9E70921E7E746210548FFF7ACFDE5E7BD
:10283400282B0008DC03002030290008F4030020C2
:10284400382C00083A289ABF0B4B1B564FF0FF3325
:10285400C3F30312052A98BF084803F00F0398BF77
:1028640050F82220064888BF002250F8233009B1CE
:10287400936170471B04FBE7282B00080C00002021
:10288400E82B0008FFF7A8BB38B5044648B1FFF7AA
:10289400A3FB0546FDF7CCFFFFF79EFB401B8442DC
:1028A400F8D838BD0B460146184600F001B80000C0
:1028B40010B5054C13462CB10A4601460220AFF36D
:1028C400008010BD204610BD0000000070B50D4E04
:1028D4000D4CA41BA4100025A54209D10B4E0C4C91
:1028E40000F018F8A41BA4100025A54205D170BD62
:1028F40056F8253098470135EEE756F825309847C5
:102904000135F2E79C2C00089C2C00089C2C000844
:10291400AC2C0008F8B500BFF8BC08BC9E46704754
:0C292400F8B500BFF8BC08BC9E46704728
:1029300000000000000C00401282000001000000B6
:10294000000C00401202010002000000000C0040D8
:102950001282010003000000000C0040120202007D
:102960000500000000000040128100000600000089
:102970000004004012820000070000000004004034
:102980001202010008000000000001401281000056
:102990000900000000000140120101000A000000CF
:1029A00000000140128101000B0000000000014006
:1029B000120102000F000000000000401281000020
:1029C000100000000004004012820100110000000D
:1029D000000400401202020013000000000000404A
:1029E00012010100140000000004004012820000E7
:1029F0001500000000040040120201001600000053
:102A0000000800401282000017000000000800408B
:102A100012020100180000000008004012820100AC
:102A20001900000000080040120202001A00000015
:102A300000000040128101001D0000000000014064
:102A4000128110001E000000000001401201110060
:102A50001F0000000000014012811100260000004C
:102A60000004004012820000270000000004004023
:102A70001202010028000000000400401282010040
:102A8000290000000004004012020200FF000000C4
:102A900000000000000000000300000000440040AF
:102AA000120700000A000000001001401207000099
:102AB0000C00000000140140120800001700000084
:102AC0000010014012070000270000000014014020
:102AD00012080000FF0000000000000000000000DD
:102AE000020000000044004012070000090000003E
:102AF00000100140120700000B000000001401400C
:102B0000120800001600000000100140120700002B
:102B1000260000000014014012080000FF00000021
:102B2000000000000000000003020A1315141A0838
:102B300009271607060519182A2CFF0D0E0F172D49
:102B40002E2F505122232B32292826250C0B1C1BFB
:102B500012111F1E1D24000104102120070622232C
:102B60002511240000000000000000006506000898
:102B70004D070008110600083B0600082106000862
:102B8000A5060008A3070008CD07000804080C2FBD
:102B9000686F6D652F6A696D6D792F2E617264752E
:102BA000696E6F31352F7061636B616765732F5389
:102BB000544D33322F68617264776172652F73747C
:102BC0006D33322F312E352E302F636F7265732F98
:102BD00061726475696E6F2F73746D33322F706913
:102BE0006E6D61702E6300000100000002000000A5
:102BF0000400000008000000100000002000000099
:102C00004000000080000000000100000002000001
:102C10000004000000080000001000000020000078
:102C200000400000008000000000000000000000E4
:102C300001020304060708092F686F6D652F6A6992
:102C40006D6D792F2E61726475696E6F31352F70DD
:102C500061636B616765732F53544D33322F686125
:102C60007264776172652F73746D33322F312E3534
:102C70002E302F636F7265732F61726475696E6F8A
:102C80002F776972696E675F6469676974616C2E1A
:042C900063000000DD
:082C94009CD5FF7F0100000048
:102C9C0039080008B90100083D0700089920000810
:042CAC009501000886
:102CB00000000000010000001000000000000240C1
:102CC0000004024000080240000C024000100240D4
:082CD000001C02400024F40086
:040000050800233993
:00000001FF
